:10000000830100308A003528F60003088301C6000A
:100010000408C7008B1C18280B1E17288312031313
:10002000861D1428FE3015280230A107A0158B105C
:10003000831203138C1E2E28981C232818120000EC
:10004000000018162E280530220203182E28220838
:10005000303E840083131A088000A20A47088400F7
:1000600046088300F60E760E0900213084004630E3
:10007000422020308400213042208301842E040657
:100080008001840A0406031D3F28003482077D3462
:100090009734B134CB34E534FF34193433344D3430
:1000A000673481349B34B534CF34E9348207023469
:1000B0000234023402340234023402340234023490
:1000C000023403340334033403340334820700342A
:1000D000003400340034003400340134013401347D
:1000E0000134013401340134013401348207033412
:1000F0001D34373451346B3485349F34B934D334A0
:10010000ED34073421343B3455346F3482070434E2
:100110000034013402340334043405340634073423
:0401200008340E345D
:10080000830120180F2C0430A0060F2C8301C10097
:10081000831203130C1E082C410899000800830161
:10082000201D142C8517152C8513201C192C051739
:100830000800051308008301C00140082B3E840016
:10084000831300080624C00A05304002031808007C
:100850001D2C8301350EF0393607AB00370EF03909
:100860003807AC00390EF0393A07AD00AE01AF01E0
:10087000AF0A1B2C4427A608031D8B25A6080319C5
:10088000432C44273E2C3230C200C3018F24A608DB
:10089000031908004427472C8301BB00201C2019A2
:1008A000522C1A262018402D201D08003B08AB00B2
:1008B000AC01AD01AE010730AF001B240430A0062F
:1008C0000F2CF401F5010310F30CF20C031C6F2C38
:1008D0007008F40771080318710AF5070310F00D8A
:1008E000F10D7208730403190034632C830120197D
:1008F0000F2C0130A006201C8A2CBD013D08353E7E
:10090000840083138001BD0A06303D02031C7E2C47
:10091000A3010F2C03302302031829240F2C830179
:10092000C401C501972C0000C40A0319C50A0A3086
:10093000F200F3014308F1004208F0006124750859
:100940004502031DA52C7408440203180800932CCB
:100950008301BF00A010AB003E08AC00AD01AE01AA
:10096000BB30AF001B240230C5243008A40031087E
:10097000A5001B240230C52424083006031D0800EE
:10098000310825060319A01408008301C000C10125
:10099000A20183168C16831218168517D82C0A30DC
:1009A000C200C3018F24C10A333041020318DC2C7A
:1009B00040082202031CCF2C851383168C1283124D
:1009C000181208008301201C2019E72C1A26201871
:1009D000402D201D08005730BE000030A824A01C68
:1009E00008008030A406AB015730AC002408AD00ED
:1009F0002508AE00BC30AF001B240430A0060F2C2D
:100A00008301201C2019052D1A262018402D201D99
:100A100008005830BE000030A824A01C0800023096
:100A2000A406AB015830AC002408AD002508AE0088
:100A3000BC30AF001B240430A0060F2C8301201C07
:100A40002019292DAB01AC01AD01AE018130AF0001
:100A50001B2C201D08005830BE000030A824A01C0C
:100A600008002030A406AB015830AC002408AD00CB
:100A70002508AE00BC30AF001B240430A0060F2CAC
:100A80008301BC013C0A353E840083130008F0005A
:100A90003C08353E8400700880003C0A353E8400E6
:100AA0008001BC0A05303C02031C422D26080A3A8C
:100AB000031D5C2DBA015E2D2608BA000530230205
:100AC0000318762CA30A080062308301BE000030B0
:100AD000A824A01C882D24083F39A9002108A907B3
:100AE00039302902031C762D3830A90097302902AD
:100AF0000318A901C030A4052908A404AB01623081
:100B0000AC002408AD002508AE00BC30AF001B24AB
:100B1000A011A1010800982D00304C2C03304C2C62
:100B200004304C2C01304C2C02304C2C08304C2C16
:100B3000831203132608F000EF3E03180800113E4D
:100B4000031C080005308A00A930700703188A0AC0
:100B5000820008008C2D8E2D902D922D942D962D97
:100B6000E22CBA2DEA2D002D762C002CBA2E1E2D4B
:100B7000F82E9C2F8301201C2019BF2D1A26201827
:100B8000402D201D08004F26270FC72DA80A023030
:100B9000A7072708BE002808A824A01C08001030BA
:100BA000A4062808AB002708AC002408AD002508DF
:100BB000AE00BC30AF001B242C30C2000130C3009B
:100BC0008F241B24A6080319E72D4427E22D0430A7
:100BD000A0060F2C8301201C2019EF2D1A262018A7
:100BE000402D201D08004F26270FF72DA80A0230A0
:100BF000A7072708BE002808A824A01C080020304A
:100C0000A4062808AB002708AC002408AD0025087E
:100C1000AE00BC30AF001B242C30C2000130C3003A
:100C20008F241B24A6080319172E4427122E0430E4
:100C3000A0060F2C55308301BE000030A824A01C54
:100C4000252E2012241C252E201659308312031322
:100C5000BE000030A824A01C080000308A0026082E
:100C60008620BD000F30BC00201E3B2EBD0EF03094
:100C7000BD05F030BC003C09A4053D08A404AB014F
:100C80005930AC002408AD002508AE00BC30AF00E0
:100C90001B242C30C2000130C3008F241B2C553084
:100CA0008301BE000030A824A01C5A2E2012241C50
:100CB0005A2E2016643083120313C200C3018F24FE
:100CC0005930BE000030A824A01C0800201E762E3B
:100CD000240E0F39BB0000308A003B085620A800C4
:100CE00000308A003B087620A700080024080F394E
:100CF000BB0000308A003B086620A80000308A0054
:100D00003B084620A7000800831203138501073023
:100D10009F008316850183128601F93083168600B1
:100D20008113861406151815193099001812181316
:100D300083121813831698128312181283160C123A
:100D40008C120B17831298178316981601130B1623
:100D50008B178312A1013A24A01DAB2E2108AA00F3
:100D60003230C200C3018F242A082106031DAB2E96
:100D70006425AB2E8301201C2019E12E4F26270F5E
:100D8000C22EA80AA70A2708BE002808A824A01C6B
:100D900008001030A4062808AB002708AC0024087F
:100DA000AD002508AE00BC30AF001B242C30C200C3
:100DB0000130C3008F241B24A60803190800442710
:100DC000DC2E201D08005830BE000030A824A01CD6
:100DD00008004030A406AB015830AC002408AD0038
:100DE0002508AE00BC30AF001B240430A0060F2C39
:100DF0008301201C2019282FAB01AC01AD01AE01ED
:100E00000330AF001B240530C5241E25C830C200A6
:100E1000C3018F243408AB00AC01AD01AE01073033
:100E2000AF001B241B24C830C200C3018F2430082C
:100E3000AB003108AC003208AD003308AE00AF01A2
:100E4000AF0A1B241B24C830C200C3018F241E2DEF
:100E5000201D08005830BE000030A824A01C080047
:100E60008030A406AB015830AC002408AD00250842
:100E7000AE00BC30AF001B240430A0060F24F430B9
:100E8000C2000130C3008F2C8301A601060E0F396A
:100E90000F3A0319992F07308504061A512F0B308A
:100EA000A600861A552F0730A600061B592F0430BE
:100EB000A600861B5D2FA601A60AF03085050B3023
:100EC0008504061A652F0A30A600861A692F083095
:100ED000A600061B6D2F0530A600861B712F023061
:100EE000A600F03085050D308504061A792F0C30E8
:100EF000A600861A7D2F0930A600061B812F06301A
:100F0000A600861B852F0330A600F03085050E3025
:100F10008504061A8D2F1030A600861A912F0F30E7
:100F2000A600061B952F0E30A600861B992F0D30AC
:100F3000A600F030850508008301201C2019B72F7A
:100F40007A30BE000030A824A01C08008030A4061F
:100F5000AB017A30AC002408AD002508AE00BC30EF
:100F6000AF001B24A608031908004427B22F201D38
:100F70000800AB01AC01AD01AE010330AF001B2492
:100F80000530C5243408BB000830AB00AC01AD010E
:100F9000AE010730AF001B240130C524AB01AC010A
:100FA000AD01AE010830AF001B240130C524A608F6
:100FB0000319DC2F4427D72FBC011E30C200C30108
:100FC0008F244427BC0AFB303C020318EA2FA608F2
:100FD0000319DD2FAB01AC01AD01AE018830AF00CC
:100FE0001B240130C5243B08AB00AC01AD01AE01B0
:100FF0000730AF001B240130C5240430A0060F2C9D
:02400E00383F39
:00000001FF
